:100000000C9465040C9482040C9482040C94820475
:100010000C9431070C9482040C9482040C94820496
:100020000C9482040C9482040C9482040C94820438
:100030000C9482040C94F7050C9482040C948204B2
:100040000C9482040C9482040C9482040C94820418
:100050000C948204204B422F73000D0A00746D3AF9
:100060002074657374206D6F6465202020200074F7
:10007000703A2075647020706F72742020202020E8
:100080000074693A2069702061646472657373203A
:1000900020200074743A207061636B657420747959
:1000A0007065202000746C3A207061636B65742069
:1000B0006C656E2020200066633A20666C6F7720A6
:1000C000636F6E74726F6C200066643A2066756CA4
:1000D0006C206475706C65782020006D3A206D612D
:1000E000632061646472657373202020001A11AF6D
:1000F000A047110000EA05FDFFC0A802DE901A002B
:1001000020202B7265713D0020763D0020643D006B
:10011000206E3D005D204552523A005D206F6B001D
:100120005B52583A005B54583A003F3F20455252C8
:100130003A00636D643D0046545064617400465457
:100140005063746C00424F4F54504300424F4F5421
:100150005053002C61636B3D002C7365713D002C86
:10016000666C6167733D005B5443503A005B5544D5
:10017000503A002C55445020002C54435020002C61
:1001800049434D50005B4950343A005245504C00B1
:1001900052455120005B4152503A003F00747800B4
:1001A00072782070696F00727820706C6970626F6D
:1001B0007800636E7420206279746573202020209B
:1001C000657272202064726F7020726174650D0A0E
:1001D00000E101CA10C50F7710F90FC7109611E1A1
:1001E0000F656E6332386A36300070696F3A206589
:1001F0007869740D0A004552524F523A00207265D8
:10020000763D0020666C6167733D003A206F6B217C
:10021000206D61633D0070696F3A20696E69743AC0
:100220002000D1015544503A2000415250205245FF
:10023000504C59210D0A00415250205245513A204C
:1002400049503D004552524F523D00206E3D0076D0
:100250003D0070696F2074783A20004552524F5229
:100260003D00206E3D00763D0070696F2072783A47
:1002700020005B50494F5F544553545D206F6666C4
:100280000D0A005B50494F5F544553545D206F6E1B
:100290000D0A006F6666006F6E005B4155544F5D3E
:1002A0002000544F54414C204552524F525320008D
:1002B0004552523A20646174612040004552523ADE
:1002C00020706B7420747970650D0A004552523AA3
:1002D00020737263206D61630D0A004552523A200B
:1002E000647374206D61630D0A004552523A2073A5
:1002F000697A650D0A005B50425F544553545D2096
:100300006F66660D0A005B50425F544553545D2092
:100310006F6E0D0A007265712069676E0D0A0052DA
:1003200045510D0A004649525354205452414E53F0
:10033000464552210D0A005B4D414749435D2072FD
:100340006571756573740D0A005B4D414749435DE6
:10035000206F66666C696E650D0A005B4D4147490A
:10036000435D206F6E6C696E650D0A005B425249F9
:100370004447455D206F66660D0A00464C4F572086
:100380006F6E0D0A00464C4F57206F66660D0A00CF
:100390004F46464C494E452044524F503A20004665
:1003A0004952535420494E434F4D494E47210D0A5F
:1003B000005B4252494447455D206F6E0D0A004E76
:1003C0004F204950563421210D0A004E4F204D41F7
:1003D00047494321210D0A005B4252494447455F8A
:1003E000544553545D206F66660D0A004F564552C2
:1003F00057524954453F210D0A005B425249444738
:10040000455F544553545D206F6E0D0A0020202037
:1004100000436F6D6D616E64204B65792048656C9B
:10042000703A0D0A00436F6D6D616E642048656C13
:10043000703A0D0A006279652E20726573746172DC
:1004400074696E672E2E2E0D0A006279650D0A0002
:100450004855483F0D0A003F3F3F0D0A00455252A4
:100460004F520D0A0053594E5441580D0A004F4B3C
:100470000D0A004F4B20284E454544205245535409
:10048000415254290D0A0052455345540D0A003E6D
:100490002000436F6D6D616E64204D6F64652E208A
:1004A000456E746572203C3F3E2B3C7265747572DC
:1004B0006E3E20666F722068656C7020616E6420ED
:1004C0003C713E2B3C72657475726E3E20746F20D9
:1004D0006C656176652E0D0A00302E362032303183
:1004E00035303131370D0A00F106CF18DF06DD0651
:1004F000D118CB06C906B419B206B006B0199F06CA
:100500009C06A81982067F06A019630660069C193E
:1005100044064106981931062E0694191D061B063D
:100520007119FF05FC052B19E305E0052B19CA0518
:10053000C705F318B005AD05F31894059105D31858
:100540007C057905F318670564052B19540500002F
:100550000000000074657374206D6F6465205B306B
:100560007C315D00746D00746573742055445020B7
:10057000706F7274203C6E3E00747000746573740A
:100580002049502061646472657373203C69703E39
:100590000074690074657374207061636B65742006
:1005A0006574682074797065203C6E3E0074740038
:1005B00074657374207061636B6574206C656E671D
:1005C0007468203C6E3E00746C0073657420666C29
:1005D0006F7720636F6E74726F6C205B6F6E5D005F
:1005E0006663007365742066756C6C206475706C4E
:1005F00065206D6F6465205B6F6E5D006664006DE5
:1006000061632061646472657373206F6620646542
:1006100076696365203C6D61633E006D00726573B1
:1006200065742073746174697374696373007372A1
:100630000064756D70207374617469737469637399
:1006400000736400726573657420706172616D651A
:100650007465727320746F2064656661756C7400D4
:100660007072006C6F616420706172616D65746599
:1006700072732066726F6D20454550524F4D007069
:100680006C007361766520706172616D657465726E
:100690007320746F20454550524F4D0070730070A9
:1006A00072696E7420706172616D65746572730039
:1006B00070007072696E74206669726D7761726520
:1006C0002076657273696F6E007600736F667420B2
:1006D0007265736574206465766963650072007184
:1006E00075697420636F6D6D616E64206D6F6465F4
:1006F0000071004F46460D0A004F4E0D0A00564548
:1007000052424F53453A200031C2191E0832C519D2
:10071000070833BE19F30734BA19E00773E919D093
:100720000753E719BF0776D119A90770CE198807B3
:1007300050CB195E0761C9193F0700000000007423
:100740006F67676C65206175746F2073656E6420D8
:1007500028706274657374206D6F64652900736519
:100760006E6420612074657374207061636B6574BE
:10077000202873696C656E74292028706274657313
:1007800074206D6F6465290073656E642061207448
:10079000657374207061636B657420287062746582
:1007A0007374206D6F64652900746F67676C6520D2
:1007B000766572626F7365206F7574707574007200
:1007C000657365742073746174697374696373000D
:1007D00064756D70207374617469737469637300F8
:1007E000656E7465722050422074657374206D6F5D
:1007F000646500656E7465722050494F207465739E
:1008000074206D6F646500656E7465722062726934
:100810006467652074657374206D6F646500656E30
:1008200074657220627269646765206D6F6465002B
:10083000726573657474696E672E2E2E0D0A0050F2
:1008400072657373203C72657475726E3E20746FAE
:1008500020656E74657220636F6D6D616E64206DCE
:100860006F6465206F72203C3F3E20666F72206B84
:1008700065792068656C700D0A006279206C616C86
:100880006C6166612028687474703A2F2F777777CF
:100890002E6C616C6C6166612E64652F626C6F6793
:1008A000290D0A0D0A000D0A57656C636F6D6520EE
:1008B000746F20706C6970626F7820302E36203231
:1008C000303135303131370D0A0011241FBECFE5EC
:1008D000D8E0DEBFCDBF10E0A0E6B0E0E0E6F5E393
:1008E00002C005900D92A03AB107D9F727E0A0EA1F
:1008F000B0E001C01D92AB34B207E1F70E94EB19E2
:100900000C94281A0C94000008958A3010F4805D2D
:100910000895895C08951F93CF93DF93182FEB01FF
:1009200082958F700E9485048883812F8F700E942A
:1009300085048983DF91CF911F9108951F93CF93F1
:10094000DF93182FEB01892F0E948B04BE016E5F8D
:100950007F4F812FDF91CF911F910C948B04CF9209
:10096000DF92EF92FF92CF93DF936B017C01EA015C
:10097000BA01C7010E949E04BE016C5F7F4FC60191
:10098000DF91CF91FF90EF90DF90CF900C949E0479
:10099000FB0164E60E94661A805D8083892F6AE00D
:1009A0000E94661A805D8183905D92830895AF9264
:1009B000BF92CF92DF92EF92FF920F931F93CF934C
:1009C000DF93EA01B22EE22FF0E03197CE0FDF1F66
:1009D000021708F4219610E02EE2A22E3AE0C32E70
:1009E000D12CE12CF12C1B1579F0101302C0A88238
:1009F0002197A70196010E94721A605D6883219772
:100A0000B901CA011F5FEFCFDF91CF911F910F9105
:100A1000FF90EF90DF90CF90BF90AF900895FB01D3
:100A20009FE9980F963010F4875509C09FEB980FF7
:100A3000963010F4875303C080538A3018F48083B3
:100A400081E0089580E00895EF92FF920F931F9345
:100A5000CF93DF931F92CDB7DEB77C018B01BE0130
:100A60006F5F7F4FFC0180810E940F05811102C0E2
:100A700080E011C089818295807F8983B801F70168
:100A800081810E940F05882399F3F8018081998163
:100A9000892B808381E00F90DF91CF911F910F917F
:100AA000FF90EF900895EF92FF920F931F93CF93D3
:100AB000DF9300D0CDB7DEB78C017B01BE016E5F46
:100AC0007F4F0E942405811102C080E013C0BE0147
:100AD0006F5F7F4FC80102960E9424058823A9F307
:100AE0008A8190E0982F88272981822BF7019183B2
:100AF000808381E00F900F90DF91CF911F910F9134
:100B0000FF90EF900895EF92FF920F931F93CF9372
:100B1000DF9300D000D0CDB7DEB77C018B01BE01E2
:100B20006C5F7F4F0E942405811102C080E02EC0BF
:100B3000BE016D5F7F4FC70102960E942405882386
:100B4000A9F3BE016E5F7F4FC70104960E94240582
:100B5000882361F3BE016F5F7F4FC70106960E9435
:100B60002405882319F32C818B8190E0A0E0B0E06C
:100B7000DC0199278827B22B2981822B2A81922B8D
:100B8000F80180839183A283B38381E00F900F905B
:100B90000F900F90DF91CF911F910F91FF90EF90E9
:100BA0000895FC0180E020E0919190539A3048F440
:100BB0003AE0239F900D1124292F8F5F8330A1F7F6
:100BC00002C0882311F0FB0120830895F8941AB81D
:100BD00010BC80E189B988E98AB986E880BD78943B
:100BE0001092A2001092A1001092A00008951F92EE
:100BF0000F920FB60F9211248F93EF93FF938CB146
:100C0000E091A100F0E0ED55FF4F80838091A100BD
:100C10008F5F8093A1008091A100803111F4109228
:100C2000A1008091A0008F5F8093A000FF91EF91C1
:100C30008F910F900FBE0F901F9018952091A200DA
:100C40009091A10081E0291301C080E00895909166
:100C5000A2008091A1009817D1F3F894E091A2002E
:100C6000F0E0ED55FF4F80819091A2009F5F90933F
:100C7000A2009091A200903111F41092A2009091E4
:100C8000A00091509093A000789408955D9BFECFB2
:100C90008CB90895CF93DF93EC01FE0184918823F2
:100CA00021F00E9446062196F8CFDF91CF9108955A
:100CB000CF93DF93EC018991882319F00E944606B7
:100CC000FACFDF91CF910895EF92FF921F93CF93C8
:100CD000DF931F92CDB7DEB7182F7C018E2D811BBD
:100CE000861740F4F70181917F0169830E944606CF
:100CF0006981F4CF0F90DF91CF911F91FF90EF901A
:100D000008958AE590E00C944A0680E20C94460629
:100D10000F936091BF007091C0008091C1009091CD
:100D2000C20004E02AE043EB50E00E94D70480E2D6
:100D30008093BE006CE083EB90E00F910C9464060E
:100D40000F9304E02AE043EB50E00E94D70480E2D6
:100D50008093BE006CE083EB90E00F910C946406EE
:100D60000F93BC0180E090E002E026E043EB50E00E
:100D70000E94D70467E083EB90E00E94640684E55C
:100D800090E00F910C944A060F93DC01CB01009781
:100D900021E0A207B10538F021E22093B30064EB13
:100DA00070E0CD010BC0803127E29207A105B105AB
:100DB00040F02EE32093B30064EB70E00E949E04A9
:100DC0000BC02BE22093B30004E024E044EB50E09E
:100DD000BC01CD010E94D70465E083EB90E00F9148
:100DE0000C94640663EB70E00E948B0462E083EB7A
:100DF00090E00C94640663EB70E00E949E0464E053
:100E000083EB90E00C94640643EB50E00E94AF0447
:100E100068E083EB90E00C946406F8948AE085BD6A
:100E200087EC83BD14BC89B7806889BF1FBC83E091
:100E30008EBD1DBC1CBC1092C6001092C500109245
:100E4000C4001092C3001092BF001092C000109214
:100E5000C1001092C2001092C8001092C70078948E
:100E600008951F920F920FB60F9211242F938F9314
:100E70009F93AF93BF938091C5009091C600019658
:100E80009093C6008093C5008091BF009091C000F0
:100E9000A091C100B091C2000196A11DB11D809327
:100EA000BF009093C000A093C100B093C200809196
:100EB000C7009091C8000196883E23E0920729F070
:100EC0009093C8008093C7000DC01092C800109284
:100ED000C7008091C3009091C40001969093C40014
:100EE0008093C300BF91AF919F918F912F910F90ED
:100EF0000FBE0F901F9018951092C4001092C3005F
:100F00002091C3003091C40028173907C8F3089511
:100F10001092C6001092C5002091C5003091C60005
:100F200028173907C8F30895FB013097A9F0DC01B1
:100F300020EA36E841E050E00E94941A9F0140E028
:100F400050E0E2E0220F331F441F551FEA95D1F70E
:100F50000E94721AC901089580E090E008958A986D
:100F6000929AD398DB9AD19AD998D298DA9AD09A51
:100F7000D89A14BA08958FEF84BB089514BA0895CF
:100F8000D8988A95F1F7D89A08951092C6001092D1
:100F9000C50020916000309161004091C5005091E2
:100FA000C6004217530780F499B392FB992790F932
:100FB000882319F0992319F00AC0992341F0CB999D
:100FC000ECCF862F83600895862F8260089581E09C
:100FD00008959093E4008093E3007093E20060939F
:100FE000E1005093E0004093DF003093DE00209357
:100FF000DD000E94BE07D998089580B329B399B344
:10100000947082FB882780F923FD826091118460AF
:10101000089581E00E94C0078091BF009091C000B8
:10102000A091C100B091C2008093D9009093DA00E2
:10103000A093DB00B093DC0008955F926F927F92E3
:101040008F929F92AF92BF92CF92DF92EF92FF92D8
:101050000F931F93CF93DF9300D01F92CDB7DEB7CE
:101060001092C900CB9904C01092CA0080E006C259
:10107000CA99FACF53B21A82198282E2581619F02D
:1010800094E4591215C06091DD007091DE00E0918A
:10109000E300F091E400AE014F5F5F4F8091DF000D
:1010A0009091E0000995813019F08093CA00E6C163
:1010B000C090BF00D090C000E090C100F090C2008E
:1010C0001DBC1CBCD99AE2E25E1681F0E51528F041
:1010D000F1E15F1609F45EC06AC183E3581609F4B2
:1010E0000EC194E4591609F4ABC061C189809A809D
:1010F00060E281E00E94C507282F813009F050C1CD
:101100000E94BB0795BAD99860E380E00E94C507AA
:10111000282F813009F044C185BAD99A80FE03C0D6
:10112000EFEF8E1A9E0A969487946090DF0070907D
:10113000E000A12CB12C8501000F111FA814B904E7
:1011400001F160E481E00E94C507282F8130F1F4AD
:10115000F301808185BBD99860E480E00E94C507D7
:10116000282F813019F00F5F1F4F10C0F3018181CC
:1011700085BBD99AFFEFAF1ABF0A82E0680E711CD7
:10118000DACF60E581E00E94C507282F2B830E94FB
:10119000BE07B3C060E281E00E94C507282F8130FE
:1011A00009F0FEC013B3D99860E380E00E94C50740
:1011B000282F813009F0F4C063B2D99A712C712ABA
:1011C0008091DD009091DE008615970508F4EBC054
:1011D00060FE03C09FEF691A790A76946794809045
:1011E000DF009090E000A12CB12C8501000F111FB1
:1011F000A614B70409F4DEC060E481E02B830E94EA
:10120000C5072B818130D1F483B3F4018083D99851
:1012100060E480E02B830E94C5072B81813019F0A8
:101220000F5F1F4F0BC083B3F4018183D99AFFEF87
:10123000AF1ABF0A82E0880E911CD7CF282FBAC000
:1012400009811A8160E281E00E94C507282F813060
:1012500009F0A6C00E94BB0715BBD99860E380E0E7
:101260000E94C507282F813009F09AC005BBD99A82
:1012700060E481E00E94C507282F813009F090C00A
:10128000C801019696958795E091DF00F091E00006
:10129000F894D99800E010E036E00817190749F0F3
:1012A000432F4A95F1F7408145BBCA9B04C0CB99B7
:1012B000FCCF789410C0432F4A95F1F7418145BB8C
:1012C000CA9903C0CB99FCCFF4CF32960F5F1F4F62
:1012D000E4CFCB9BEECFCA99FCCFD99ACA9903C071
:1012E000CB99FCCFE6CF0817190708F422E4D99868
:1012F0002B830E94BE07000F111F2B815BC060E291
:1013000081E00E94C507282F813009F049C013B33E
:10131000D99860E380E00E94C507282F813009F04A
:101320003FC083B390E0912B4091DD005091DE00EF
:1013300048175907C0F10196969587954091DF00AF
:101340003091E000F894D99AE42FF32F00E010E0F8
:101350000817190721F4789413C0CB9BFCCFCA9BC4
:10136000FCCF33B33083CA9B03C0CB99FCCFF3CF00
:1013700033B331830F5F1F4F3296EACFCB9BEBCF56
:10138000CA9BFCCFD998CA9B03C0CB99FCCFE3CFB3
:101390000817190708F422E4D99A000F111F0AC090
:1013A00000E010E007C000E010E025E003C000E02E
:1013B00010E024E01092C6001092C50080916000F9
:1013C000909161004091C5005091C600481759079F
:1013D00010F4CB99F7CFD998ACB4BDB4213089F4CF
:1013E00091E1591619F0E3E35E120BC0E091E100C0
:1013F000F091E200B8018091DF009091E000099542
:10140000282F5092C9002093CA001093CE00009359
:10141000CD00B092D000A092CF00B501C8012B83BF
:101420000E9494079093D2008093D100C092D5007F
:10143000D092D600E092D700F092D8002B81F1E153
:1014400081E05F1619F093E3591280E08093CB009E
:101450008093CC0081110BC08091D5009091D60073
:101460004091D9005091DA00841B950B02C080E0B6
:1014700090E09093D4008093D300822F0F900F9030
:101480000F90DF91CF911F910F91FF90EF90DF9020
:10149000CF90BF90AF909F908F907F906F905F9014
:1014A00008958FEF9FEFEFECF6E021918227282F30
:1014B00022952827022E269526952025022E269550
:1014C00020252770082E892F269507942795902D83
:1014D0008227069427959025822726E0E23EF20790
:1014E00021F70895CF93DF938BED90E00E944A0699
:1014F0008FEC96E00E94580B0E9481060E948106A4
:10150000C091D60689EC90E00E944A068C2F0E947A
:10151000F2060E948106C091D50687EB90E00E94FA
:101520004A068C2F0E94F2060E9481060E948106C4
:10153000C091D706D091D80685EA90E00E944A066D
:10154000CE010E94FB060E948106C091D906D0916F
:10155000DA0683E990E00E944A06CE010E94FB066B
:101560000E94810681E890E00E944A068BED96E099
:101570000E94CF0B0E948106C091DF06D091E00649
:101580008FE690E00E944A06CE010E94FB060E9470
:101590008106C091E1068DE590E00E944A068C2FFD
:1015A0000E94F206DF91CF910C948106E19911C05F
:1015B00043E150E062E070E08FEC96E00E944A1A4E
:1015C0000E94510ABC0180E090E00E94611A80E014
:1015D000089581E00895AFECB6E0EDEEF0E084917F
:1015E0008D93319681E0E030F807C9F70895CF93E5
:1015F000DF93E19916C043E150E062E070E08FECC8
:1016000096E00E94341A80E090E00E94441AEC01B7
:101610000E94510AC817D90731F00E94EB0A82E0F4
:1016200003C081E001C080E0DF91CF9108950E9466
:10163000F70A81110C94EB0A0895FB0120E030E0D9
:10164000DC014D91CD0141932F5F3F4F2630310595
:10165000B9F70895FB0120E030E0DC014D91CD01A8
:1016600041932F5F3F4F24303105B9F70895FC01B6
:10167000808190E0982F88272181822B0895FC019A
:10168000708361830895FC0120816181862F90E041
:10169000A0E0B0E077276627922B2381622B22817E
:1016A000722B0895FC0170836183528343830895F4
:1016B0000F931F93CF93DF938C01CEE7D0E0BE0151
:1016C000F80181918F010E948B042396F0E0C039CC
:1016D000DF07A9F78EE790E0DF91CF911F910F917F
:1016E0000C945806CF92DF92EF92FF920F931F93C4
:1016F000CF93DF931F92CDB7DEB77C016B0100E083
:1017000010E0BE016F5F7F4FC7010E94D1058823A3
:1017100071F090E00196E80EF91E8981F60181933F
:101720006F010F5F1F4F0430110559F781E00F90D3
:10173000DF91CF911F910F91FF90EF90DF90CF90AD
:101740000895CF92DF92EF92FF920F931F93CF9362
:10175000DF931F92CDB7DEB77C016B0100E010E094
:10176000BE016F5F7F4FC7010E942405882369F087
:1017700083E0E80EF11C8981F60181936F010F5F10
:101780001F4F0630110561F781E00F90DF91CF9177
:101790001F910F91FF90EF90DF90CF9008950F93DE
:1017A0001F93CF93DF938C01C0E9D0E0BE01F80115
:1017B00081918F010E94C8042496F0E0C03ADF07AF
:1017C000A9F780E990E0DF91CF911F910F910C94E0
:1017D0005806FB0120E030E0DC015D91CD01419134
:1017E000541307C02F5F3F4F26303105A9F781E022
:1017F000089580E00895FB0120E030E0DC015D9178
:10180000CD014191541307C02F5F3F4F2430310564
:10181000A9F781E0089580E008950F931F93CF9377
:10182000DF93EC016C317105A0F00E94370B8C0145
:10183000CE0102960E94370B3C812D8101301105AB
:1018400041F48115984029F4363019F481E02430B0
:1018500009F080E0DF91CF911F910F910895AF9231
:10186000BF92CF92DF92EF92FF920F931F93CF938D
:10187000DF93EC016B015A0162E070E006960E9472
:101880003F0B7E0188E0E80EF11CBE016E5E7F4FCB
:10189000C7010E941D0B8E01025F1F4FBE01685ED3
:1018A0007F4FC8010E942A0BB701C6010E941D0B81
:1018B000B801C501DF91CF911F910F91FF90EF907B
:1018C000DF90CF90BF90AF900C942A0BCF93DF9313
:1018D000EC018334910519F48CE491E005C0843463
:1018E000910531F485E491E0DF91CF910C944A06A3
:1018F00080E20E944606CE010E94FB0680E2DF9154
:10190000CF910C944606CF93DF93EC01853191057E
:1019100019F48EE391E005C08431910531F487E339
:1019200091E0DF91CF910C944A0680E20E94460636
:10193000CE010E94FB0680E2DF91CF910C94460617
:10194000EF92FF920F931F93CF93DF9300D000D0BD
:10195000CDB7DEB77C018B018BE50E944606B8014E
:1019600080E090E004E024E0AE014F5F5F4F0E9412
:10197000D70464E0CE0101960E9464068CE20E94C6
:101980004606C7010C960E94370B0E94FB068CE2AC
:101990000E944606C70106960E94580B8EE30E94DD
:1019A0004606C7010E94580B8DE50E94460680E25C
:1019B0000E9446060F900F900F900F90DF91CF91ED
:1019C0001F910F91FF90EF900895CF93DF93EC015B
:1019D00085E991E00E944A06CE0106960E94370BE7
:1019E0008130910519F480E991E005C082309105BC
:1019F00029F48BE891E00E944A0602C00E94FB068F
:101A00008CE20E94460688E20E944606CE010896B5
:101A10000E94580B8CE20E944606CE010E960E9450
:101A2000CF0B89E20E9446068EE30E94460688E2BA
:101A30000E944606CE0142960E94580B8CE20E94FC
:101A40004606CE0148960E94CF0B89E20E944606C8
:101A50008DE50E94460680E2DF91CF910C94460608
:101A60001F93CF93DF93EC0185E891E00E944A0633
:101A70008A8190E0982F88272B81822B0E94FB0679
:101A80001985113019F48FE791E004C0163029F45C
:101A900089E791E00E944A060CC0113119F483E7EE
:101AA00091E0F8CF8CE20E944606812F90E00E94E0
:101AB000FB068CE20E944606CE010C960E94CF0BDC
:101AC0008EE30E944606CE0140960E94CF0B8DE524
:101AD0000E94460680E2DF91CF911F910C9446064A
:101AE000CF92DF92EF92FF92CF93DF93FC012081A0
:101AF0002F70220F220F7C01E20EF11C81858131B3
:101B0000B9F48DE691E00E944A06C7010E94370BA6
:101B10006C01C70102960E94370BEC01C6010E94BE
:101B2000660C8EE30E944606CE010E94660C40C001
:101B3000863009F049C087E691E00E944A06C70155
:101B40000E94370BEC01C70102960E94370B6C0113
:101B5000CE010E94830C8EE30E944606C6010E94BD
:101B6000830CC7010C960E94370B6C018FE591E046
:101B70000E944A06C60191700E94FB0689E591E029
:101B80000E944A06C70104960E94430B0E94040764
:101B9000C4FE0EC0C70108960E94430B6B017C0176
:101BA00083E591E00E944A06C701B6010E9404073E
:101BB0008DE50E94460680E2DF91CF91FF90EF9085
:101BC000DF90CF900C944606DF91CF91FF90EF907D
:101BD000DF90CF9008950F931F93CF93DF938C01E5
:101BE0000E94A00CE8012E96C8010C960E94370BAB
:101BF000863028E0920739F4CE01DF91CF911F9112
:101C00000F910C94E50C8115984051F4CE010E947F
:101C1000300DCE01DF91CF911F910F910C94700D7B
:101C2000DF91CF911F910F910895EF92FF920F9343
:101C30001F93CF93DF9300D000D0CDB7DEB77C01E8
:101C40000E948806F7011081123241F018F4113118
:101C500039F404C0133311F0143411F481E001C0DD
:101C600080E0F701018181110FC082E391E00E94C1
:101C70004A06812F0E94F2068AE291E00E944A06FB
:101C8000802F0E94F2065DC0F7018281882319F03F
:101C900085E291E002C080E291E00E944A06812F35
:101CA0000E94F206013029F48BE191E00E944A067D
:101CB00007C084E191E00E944A06802F0E94F2064C
:101CC00080E191E00E944A06F7016481758180E01D
:101CD00090E004E024E0AE014F5F5F4F0E94D70424
:101CE00064E0CE0101960E9464068CE091E00E94BF
:101CF0004A06F7016681778180E090E024E0AE013A
:101D00004F5F5F4F0E94D70464E0CE0101960E94AE
:101D1000640688E091E00E944A06F701808591857B
:101D20000E94B006F701828181110BC080E091E032
:101D30000E944A06F7016285738580E090E00E9468
:101D4000C4060E9481060F900F900F900F90DF91B4
:101D5000CF911F910F91FF90EF900895FF920F93F5
:101D60001F93CF93DF93F82E082F10E08CE0F89E9E
:101D7000E0011124CE51D94F8C819D810E94FB0638
:101D80000E948506688179818A819B810E9404076F
:101D90000E9485068E819F810E94FB060E94850617
:101DA000888599850E94FB060E9485068A859B8509
:101DB0000E94B0060E94850683E08F1540F0F8016E
:101DC000EE0FFF1FEA58FF4F8081918102C08BE91F
:101DD00091E00E944A06DF91CF911F910F91FF90F1
:101DE0000C948106E2EEF6E01082118212821382D8
:101DF0001582148217821682118610861386128627
:101E00003C9687E0E231F80779F708950F931F9326
:101E10009CE0899FF0011124EE51F94F8481958156
:101E20000196958384830081118122813381060F7D
:101E3000171F211D311D0083118322833383828567
:101E400093858417950710F4538742871F910F914C
:101E5000089582EB91E00E944A0680E00E94AE0E57
:101E600081E00E94AE0E82E00E94AE0E83E00C94F0
:101E7000AE0ECF93DF93D82FC62F82EB91E00E9456
:101E80004A06DD2331F080E00E94AE0E81E00E9420
:101E9000AE0ECC2341F082E00E94AE0E83E0DF91D3
:101EA000CF910C94AE0EDF91CF91089587B3806BE4
:101EB00087BBBE9888B38F7588BBC49A80E58DB9FF
:101EC00081E08EB90895C4986F71682B6FB9779BC4
:101ED000FECF4FB9779BFECFC49A0895C4982AE3EA
:101EE0002FB9779BFECFFB01860F971FE817F907E5
:101EF00031F01FB8779BFECF2FB12193F7CFC49A53
:101F00000895CF93C82FC0766C2F70E020911607EC
:101F100030E06217730781F043E06FE180EA0E94CE
:101F2000630FC09316074C2F4295469547706FE19B
:101F300080E8CF910C94630FCF9108951F93CF93B6
:101F4000DF931F92CDB7DEB7182F69830E94810FF0
:101F50004981612F80E40F90DF91CF911F910C9404
:101F6000630F1F93CF93DF931F92CDB7DEB7182F68
:101F700079830E949E0F7981672F81E0810F0F90F6
:101F8000DF91CF911F910C949E0F8FE10E94810FE2
:101F900044E06FE180EA0C94630F60911407709144
:101FA00015076150710961158AE1780710F06FEF2C
:101FB00079E18CE00E94B10F40E46EE180E80C947E
:101FC000630F811114C080911307882321F06623C9
:101FD00039F082E006C081E0611103C080E001C0F9
:101FE00083E0682F87E70E949E0F80E0089581E0DC
:101FF0000895CF92DF92EF92FF920F931F93CF93AA
:10200000DF9300D000D000D0CDB7DEB77C018B01CC
:102010006A01609114077091150780E00E94B10F6A
:10202000BE016F5F7F4F86E090E00E946E0F898156
:102030009A8190931507809314072B813C8124503B
:102040003109F601318320838D8187FD04C00E9410
:10205000CD0F83E00FC00217130718F08901D12CB0
:1020600002C082E0D82EB701C8010E946E0F0E9404
:10207000CD0F8D2D26960FB6F894DEBF0FBECDBFC7
:10208000DF91CF911F910F91FF90EF90DF90CF9054
:102090000895C498982F9F719FB9779BFECF87FDB5
:1020A00002C01FB804C01FB8779BFECFFACF779B42
:1020B000FECF8FB1C49A0895CF93C82F0E94810F8D
:1020C0008C2FCF910C944910CF93DF93EB01682FA5
:1020D00084ED0E949E0FBE0186ED0E94B10F8AEE34
:1020E0000E945C1080FDFBCFDF91CF910895EF92AD
:1020F000FF921F93CF93DF931F92CDB7DEB7182FB8
:102100007B0160E07AE182E099830E94B10F40E0B8
:1021100060E08AE70E94630FC4988AE78FB99981CB
:10212000779BFECFE12FF92FCF018E0D9F1DE81772
:10213000F90729F021912FB9779BFECFF8CFC49AE8
:102140008FE10E94491083FF10C08CE10E945C1057
:1021500081FFF6CF40E86FE180E80E94630F40E81E
:102160006FE180EA0E94630FEBCFB701765E86E0F5
:102170000E94B10F48E06FE180E80E94630F80E0A9
:102180000F90DF91CF911F91FF90EF90089589E319
:102190000C945C10FF920F931F93CF93DF93EC018D
:1021A000F62E0E94560FC49A8F2D817080931307CC
:1021B0004FEF60E08FEF0E94630F8FE39FE1019785
:1021C000F1F700C000000FEF1FE08DE10E94491001
:1021D000811107C00150110901151105B1F781E006
:1021E0009FC0109215071092140760E070E088E01D
:1021F0000E94B10F60E070E08CE00E94B10F6FEFC1
:1022000079E18AE00E94B10F60E07AE184E00E9407
:10221000B10F6FEF7FE186E00E94B10FF2FE02C0C6
:1022200061EA01C060EA88E30E949E0F6FE370E3F9
:1022300088E20E94B10F69EF77EF80E30E94B10F4F
:102240006DE080EC0E949E0F60E081EC0E949E0F8A
:1022500010911307111102C062E301C063E382EC25
:102260000E949E0F112339F065E184EC0E949E0FBD
:1022700062E170E006C062E184EC0E949E0F62E1C0
:102280007CE086EC0E94B10F6EEE75E08AEC0E9455
:10229000B10F112341F060E071E080E00E94641012
:1022A00060E070E007C060E070E080E00E946410D1
:1022B00060E071E080E10E94641060ED77E088E703
:1022C0000E94B10F82E70E945C10863008F08F5F99
:1022D00080931207688184EE0E949E0F698185EECB
:1022E0000E949E0F6A8182EE0E949E0F6B8183EE98
:1022F0000E949E0F6C8180EE0E949E0F6D8181EE88
:102300000E949E0F8FE10E94810F40EC6BE180E8FC
:102310000E94630F44E06FE180E80E94630F80E059
:10232000DF91CF911F910F91FF900895CF93DF938D
:10233000EB01882359F08130F1F461E184ED0E94D2
:102340009E0F61E082ED0E949E0F03C080911207F4
:102350000FC08AEE0E945C1080FDFBCF60E082ED32
:102360000E949E0F89ED0E945C1082FB882780F9F5
:10237000888380E002C0188281E0DF91CF910895C8
:10238000811104C01092190781E0089580E008953A
:10239000EF92FF920F931F93CF93DF931F92CDB7CE
:1023A000DEB78C01F62EE0911907F0E0EE0FFF1F6B
:1023B000EE5DFD4F859194919093180780931707D8
:1023C0000E94880686E192E00E944A06E091170783
:1023D000F0911807859194910E944A06E0911707A1
:1023E000F09118073296259134916F2DC801F901AB
:1023F0000995E82E811124C08BE092E00E944A06E4
:10240000C8010E94580B83E092E00E944A068F2D7B
:102410000E94F206E0911707F09118073C9625916B
:102420003491BE016F5F7F4F80E0F9010995E82E7E
:1024300081110DC08DEF91E00E944A06898105C08F
:1024400086EF91E00E944A068E2D0E94F2060E94BD
:1024500081068E2D0F90DF91CF911F910F91FF90EC
:10246000EF9008950E9488068AEE91E00E944A0645
:10247000E0911707F0911807349685919491FC012B
:102480000994E0911707F091180736962591349139
:10249000F9010994E0911707F091180738962591F2
:1024A0003491F9010994E0911707F09118073A96D1
:1024B00085919491FC010994E0911707F091180718
:1024C0003C9625913491F9010994E0911707F09118
:1024D00018073E9625913491F90109948091D5060B
:1024E000811102C084E001C08CE09091D606911168
:1024F00081600895FF920F931F93CF93DF93EC01B8
:102500001DBC1CBCAC016AEE75E085EE90E00E943B
:102510004A12F82E6CB57DB50990D881C02DCE0138
:102520000E9494078C01F11006C0AC01BE0182E04C
:102530000E94060F0AC020910007309101072F5F0B
:102540003F4F30930107209300078091490788236C
:1025500001F10E94880689E692E00E944A06F11085
:102560000FC086E692E00E944A06C8010E94B006AB
:1025700082E692E00E944A06CE010E94FB0607C056
:102580008BE592E00E944A068F2D0E94F2060E947F
:1025900081068F2DDF91CF911F910F91FF900895AC
:1025A000FF920F931F93CF93DF93EC011DBC1CBCD4
:1025B000BC0185EE90E00E944112F82E6CB57DB50D
:1025C000CE010E9494078C01F11006C0AC01BE013F
:1025D00083E00E94060F0AC020910C0730910D077E
:1025E0002F5F3F4F30930D0720930C0780914907D1
:1025F000882301F10E94880682E592E00E944A0643
:10260000F1100FC08FE492E00E944A06C8010E94B8
:10261000B0068BE492E00E944A06CE010E94FB06BF
:1026200007C084E492E00E944A068F2D0E94F206C1
:102630000E9481068F2DDF91CF911F910F91FF9006
:102640000895CF93DF93EC0181EF90E00E94370B68
:102650008630984009F04FC0CF30D10508F44BC008
:10266000BE016E50710983EF90E00E940D0C88232B
:1026700009F43FC089EF90E00E94370B0197C9F53C
:1026800080914907882361F00E94880687E392E0E1
:102690000E944A068BE091E00E94CF0B0E948106C7
:1026A0006BED76E08BE091E00E94FB0B882309F153
:1026B0004BED56E06FEC76E083EF90E00E942F0C3C
:1026C00065EE70E080E790E00E941D0B6BEE70E01D
:1026D0008FEC96E00E941D0BCE010E94D0128091DB
:1026E0004907882331F00E9488068AE292E00E941E
:1026F0004A0681E001C080E0DF91CF910895CF923A
:10270000DF92EF92FF920F931F93CF93DF93C091CD
:10271000F300CF70CC0FCC0FD0E0CD50DF4F8E0147
:102720000E5F1F4FC8010E94370B7C0163E071E010
:102730008BED96E00E94FB0B8823E1F18091DF0690
:102740009091E006E816F906A9F5809149078823DB
:1027500059F00E94880684E292E00E944A06888529
:102760000E94F2060E94810663E071E08FEF90E024
:102770000E942A0B6FEF70E08BED96E00E942A0B0F
:10278000CE010E94370B6C01B701CE010E943F0BB6
:10279000B601C8010E943F0B65EE70E08BEE90E041
:1027A0000E941D0B6BEE70E08FEC96E00E941D0BFB
:1027B00081E001C080E0DF91CF911F910F91FF90E8
:1027C000EF90DF90CF9008951F93CF93DF9300D0C9
:1027D000CDB7DEB70E94880683E892E00E944A06E1
:1027E0000E946E12682F8FEC96E00E94C8110E9422
:1027F000F20E10E080914A07833059F50E94971736
:10280000182F81FD26C00E945312882399F3CE0110
:1028100001960E947A12811111C089819A810E94C9
:1028200021138111E7CF89819A810E947F13882328
:1028300009F389819A810E94D012DCCF2091000790
:10284000309101072F5F3F4F30930107209300071E
:10285000D1CF61E080E00E94390F0E9432120E94C5
:10286000880682E792E00E944A06812F0F900F901F
:10287000DF91CF911F910895CF930E941D08C82F1B
:10288000882359F18130A9F44091D1005091D200B0
:102890006091CD007091CE008091CC000E94060F17
:1028A000809149078823D9F089EC90E00E94150EA9
:1028B00016C089EC90E00E94150EE091CC008CE0EF
:1028C000E89FF0011124EE51F94F268137812F5FE7
:1028D0003F4F378326838C2F03C080E001C081E007
:1028E000CF910895CF92DF92EF92FF920F931F93B3
:1028F000CF93DF938C017B018091D7069091D8060E
:102900006817790739F08AEE92E00E944A06C1E022
:10291000D0E002C0C0E0D0E060E770E0C8010E94F3
:10292000E90B811105C021968BED92E00E944A06C9
:102930006FEC76E0C80106960E94E90B811105C094
:1029400021968CEC92E00E944A068091D9069091E3
:10295000DA06F8012485291303C09585981729F014
:1029600021968CEB92E00E944A066701FEE0CF1AA6
:10297000D108025F1F4F76018C2D8E19E114F104EE
:1029800091F0F80191918F01981749F080EB92E056
:102990000E944A06C7010E94FB060E948106F1E0E0
:1029A000EF1AF108E9CF209759F082EA92E00E94ED
:1029B0004A06CE010E94FB060E94810686E001C005
:1029C00081E0DF91CF911F910F91FF90EF90DF9009
:1029D000CF9008950F931F93CF93DF93EC018A015B
:1029E0008091D7069091D806FA0191838083681769
:1029F000790720F1BE0180E790E00E941D0BBE0127
:102A00006A5F7F4F8FEC96E00E941D0B8091D90684
:102A10009091DA069C878D879E01225F3F4FF801D7
:102A2000808191818C0F9D1FF9014E2F421BE81769
:102A3000F90711F04193F9CF81E001C085E0DF9102
:102A4000CF911F910F91089580931A070C94090854
:102A500081E090911B07911180E080931B070E94F9
:102A600088068AE992E00E944A0680911B07882323
:102A700019F087E992E002C083E992E00E944A06D9
:102A80000E94810680911B07882339F081E08093A2
:102A90001A070E9409080C94F20E0895CF93DF9351
:102AA0000E94880686E093E00E944A060E94F20E89
:102AB0002AEE35E045EE50E062E774E18AEE94E1FB
:102AC0000E94E90710921B0710921C0710921A0728
:102AD000C0E0D1E080914A07823051F50E949717FB
:102AE000C82F81FD25C00E943C148130C1F4809123
:102AF0001A07811104C089EC90E00E94150E8091A4
:102B0000CB00882339F380911B07882329F0D093C9
:102B10001A070E940908DECF10921A07DBCF88231C
:102B2000C9F280911B078823A9F20E942815D2CFF1
:102B300060E081E00E94390F0E94880686EF92E0F3
:102B40000E944A068C2FDF91CF910895CF93DF9397
:102B5000EA0180911E0781FF1AC08D7F80931E07B6
:102B600065EE70E080E790E00E941D0B6BEE70E078
:102B70008FEC96E00E941D0B6FEF7FEF81EF90E0EE
:102B80000E943F0B8EE090E09983888310C0CA01B9
:102B90000E947A1280911E0782FF09C08B7F80936A
:102BA0001E070E94880685E293E00E944A06109262
:102BB0001D0781E0DF91CF91089580911D0781115C
:102BC0000EC081E080931D070E940908809149078B
:102BD000882379F00E9488068FE193E008C08091F5
:102BE0004907882331F00E94880685E193E00C9420
:102BF0004A0608950F931F93CF93DF93EC018B0147
:102C00000C960E94370B8E3F2FEF920749F130F45C
:102C1000039691F580911E0782603EC00E9488064F
:102C20008BE593E00E944A0680911E0785608093A1
:102C30001E072696BE018FEC96E00E94E90B8111DB
:102C40002FC06FEC76E0CE010E941D0B0E94D60AC9
:102C50000E94321264E08FEC96E00E94C81120C0FE
:102C60000E94880689E493E00E944A0680911E072C
:102C70008E7F80931E0714C0C8010E94D0128091DD
:102C80001E0780FD0DC00E94880687E393E00E9426
:102C90004A0680911E07866080931E070E94DD15FC
:102CA00081E0DF91CF911F910F910895DF92EF9214
:102CB000FF920F931F93CF93DF9300D0CDB7DEB772
:102CC0000E94880681EB93E00E944A062AEE35E0D6
:102CD00045EE50E06AEF75E186EA95E10E94E9076A
:102CE0000E946E12682F8FEC96E00E94C8110E941D
:102CF000F20E10921E0710921D07D090D506FF24E9
:102D0000F39410E000E080914A07811155C00E94C1
:102D10009717082F81FD50C00E943C140E94531247
:102D2000E82E882301F1FF2031F00E9488068FE908
:102D300093E00E944A0680911E0780FF03C00E9414
:102D4000DD1510C0CE0101960E947A120E948806FD
:102D500080E993E00E944A0689819A810E94FB06DD
:102D60000E948106F12CDD2071F2112391F0E11017
:102D700021C060E080E00E946512809149078823AD
:102D800031F00E94880685E893E00E944A0610E030
:102D9000BACF81E08E15D8F761E080E00E9465121D
:102DA00080914907882331F00E9488068BE793E0E1
:102DB0000E944A0611E0A7CF0E94290F0E943212FA
:102DC0000E9488068CE693E00E944A06802F0F90AE
:102DD0000F90DF91CF911F910F91FF90EF90DF90B7
:102DE0000895CF93DF93EB0181EF90E00E94370BC2
:102DF0002091E10621110CC0039619F08BEC93E0B1
:102E00000CC060E078E081EF90E00E943F0B08C0CA
:102E10008115984029F08FEB93E00E944A0603C089
:102E2000CE010E94D01281E0DF91CF9108952091D0
:102E30001F0730912007FA0131832083621773073F
:102E400078F02091E106211105C06DEF7FEF0C961F
:102E50000E943F0B1092200710921F0781E00895F7
:102E600085E008951F93CF93DF9300D0CDB7DEB7F1
:102E70000E9488068AEF93E00E944A062AEE35E017
:102E800045EE50E061EF76E187E197E10E94E907C6
:102E90000E946E12682F8FEC96E00E94C8110E946B
:102EA000F20E10E080914A07813081F50E94971759
:102EB000182F81FD2BC00E943C140E9453128823BE
:102EC00089F3CE0101960E947A128111EBCF89819C
:102ED0009A810E9421138111E5CF89819A810E94F4
:102EE0007F138823F9F220911F0730912007232BAD
:102EF00021F08CEE93E00E944A0629813A813093BA
:102F0000200720931F070E940908CCCF0E94290F99
:102F10000E9432120E94880688ED93E00E944A06C1
:102F2000812F0F900F90DF91CF911F910895AF9255
:102F3000BF92CF92DF92EF92FF920F931F93CF93A6
:102F4000DF930E941E06811102C0F12C1CC10E9459
:102F500027068A3009F0E7C082E994E00E944A0619
:102F6000E12CFF24F3948FE894E00E944A06C0E02D
:102F70000E9427068A30C1F08F3711F0883031F473
:102F8000CC23B1F3C1500E944606F2CF90EE980FC9
:102F9000903670F7EC2FF0E0E75DF84F80830E94E9
:102FA0004606CF5FCF3121F70E948106EC2FF0E07B
:102FB000E75DF84F1082CC23B1F2D12C80E0A82F2E
:102FC000B0E0A75DB84F9C91903211F48F5FF7CFBE
:102FD0009923C9F0ED2DF0E0EE0FFF1FEF5DF84FE4
:102FE000B183A083D394E82FF0E0E75DF84F9081A0
:102FF0008F5F903221F09111F6CF90E001C091E007
:1030000010829111DCCFDD2009F480C000912107EE
:1030100010912207F80180818F3369F585E294E0F1
:103020000E944A0608EE14E0F80125913491A22E80
:10303000C22FD32F209709F469C0F8013496C590A8
:10304000D490BC2EBA18FE018491882321F00E94EE
:1030500046062196F6CFF9E0FB1528F080E20E94A3
:103060004606B394F8CFC6010E944A060E94810624
:103070000A5F1F4FD9CFC8EED4E0FE01659174916D
:103080006115710509F43EC0C8010E942B1A892BF5
:1030900011F02696F2CF2097A9F12296FE012591F4
:1030A000349161E277E08D2DF9010995E82E0E94B7
:1030B000F2060E9485068E2D807FB9F4F2E0EF12B1
:1030C00007C087E894E00E944A0692E0F92E5BC0B0
:1030D00083E0E81207C083E794E00E944A0683E099
:1030E000F82E41CF8EE694E00FC0803119F485E6CA
:1030F00094E00AC0803219F48DE594E005C087E5BC
:1031000094E002C080E594E00E944A06E1E0EE12FD
:103110002ACFFE1203C08AE494E002C085E394E063
:103120000E944A0630C08F33D1F481E194E00E94BE
:103130004A06C8E0D7E0FE018491882311F1339656
:10314000059114910E9446068DE094E00E944A0683
:10315000C8010E944A060E9481062596ECCFE8E04D
:10316000F7E09491981729F0992309F4EECE35965B
:10317000F8CF309709F4E9CE319685919491FC010E
:103180000995FF24F3948F2DDF91CF911F910F911B
:10319000FF90EF90DF90CF90BF90AF90089581E0C7
:1031A000089582E00895CF93DF9300D000D0CDB78B
:1031B000DEB7FB01BE016F5F7F4F828193810E946A
:1031C000720B882341F06BED76E0CE0101960E94F0
:1031D0002A0B80E001C081E10F900F900F900F90BB
:1031E000DF91CF9108950F931F93CF93DF9300D07A
:1031F000CDB7DEB7FB01A081B18111969C911197EB
:103200002C91243701F5903739F0943741F09C36F2
:10321000D1F407ED16E005C00FED16E002C009ED90
:1032200016E0813081F0BE016F5F7F4F8281938114
:103230000E945305882339F089819A81F80191838E
:10324000808380E001C081E10F900F90DF91CF91EA
:103250001F910F9108950F931F93CF93DF9300D089
:10326000CDB7DEB7FB01A081B1812C9111969C9165
:10327000243741F49D3669F59091E10620E001EE96
:1032800016E011C0263629F5933641F0943609F53B
:103290009091D60623E006ED16E005C09091D50684
:1032A00023E005ED16E0813021F4992371F080E0F0
:1032B0000CC0BE016F5F7F4F828193812A830E9481
:1032C00024052A81882329F08981F8018083822FAF
:1032D00001C081E10F900F90DF91CF911F910F916D
:1032E0000895CF93DF9300D000D000D0CDB7DEB7E4
:1032F000FB01BE016F5F7F4F828193810E94A10B12
:10330000882341F06FEC76E0CE0101960E941D0B00
:1033100080E001C081E126960FB6F894DEBF0FBEB3
:10332000CDBFDF91CF9108950E94F20E80E0089505
:103330000E94290F80E008950E94EB0A80E0089522
:103340000E94F70A882311F08062089580E00895B2
:103350000E94D60A882311F08062089580E00895C3
:103360000E94720A80E0089589ED94E00E944A0666
:1033700080E0089582E080934A07089583E0809377
:103380004A07089510924A07089581E080934A07FA
:1033900008950C94281581E00C94241580E00C9479
:1033A000241581E090914907911180E080934907AD
:1033B0008EEF96E00E944A0680914907882319F013
:1033C00089EF96E002C083EF96E00C944A060C94D5
:1033D000F20E0C94290F0E9484040E940D070E9493
:1033E000E6050E94AF0786EA98E00E944A068AE74F
:1033F00098E00E944A060E94170B0E94720A0E94DF
:1034000081068FE398E00E944A0680914A07823045
:1034100039F0833041F0813049F40E94321708C0FE
:103420000E944E1505C00E94E41302C00E94561669
:10343000823059F780E398E00E944A062FEF81EE30
:1034400094E0215080409040E1F700C00000C3CFDD
:10345000F8940C94AE1AFB01DC018D910590801953
:103460000110D9F3990B0895DC01CB01FC01E1991E
:10347000FECF06C0FFBBEEBBE09A31960DB20D92B7
:1034800041505040B8F70895A8E1B0E042E050E064
:103490000C94361ADC01CB0103C02D910E94551A01
:1034A00041505040D0F70895262FE199FECF9FBBA1
:1034B0008EBB2DBB0FB6F894E29AE19A0FBE01962F
:1034C00008950E94541A272F0C94551A991B79E0DD
:1034D00004C0991F961708F0961B881F7A95C9F7A4
:1034E00080950895A1E21A2EAA1BBB1BFD010DC0F9
:1034F000AA1FBB1FEE1FFF1FA217B307E407F507A4
:1035000020F0A21BB30BE40BF50B661F771F881F7F
:10351000991F1A9469F760957095809590959B0115
:10352000AC01BD01CF0108950E949F1AA59F900D87
:10353000B49F900DA49F800D911D11240895A29F0A
:10354000B001B39FC001A39F700D811D1124911D77
:10355000B29F700D811D1124911D0895F894FFCF25
:103560008813FFFFFFFF00000000000000000000C4
:10357000FFFFFFFFFFFFA7019D01A0019D0130306C
:103580003A30303A30303A30303A30303A30300039
:103590003030302E3030302E3030302E3030300061
:00000001FF
